 compcie950

 Timestamp is 478248a1 (Mon Jan 07 15:43:29 2008)

 Preferred load address is 10000000

 Start         Length     Name                   Class
 0001:00000000 00000932H .rdata                  CODE
 0001:00000934 0000005dH .rdata$debug            CODE
 0001:00000994 00008fc0H .text                   CODE
 0001:00009954 00000028H .idata$2                CODE
 0001:0000997c 00000014H .idata$3                CODE
 0001:00009990 00000140H .idata$4                CODE
 0001:00009ad0 00000016H .idata$6                CODE
 0001:00009af0 00000203H .edata                  CODE
 0002:00000000 00000140H .idata$5                DATA
 0002:00000140 00000020H .data                   DATA
 0002:00000160 00000004H .bss                    DATA
 0003:00000000 00000a08H .pdata                  DATA

  Address         Publics by Value              Rva+Base     Lib:Object

 0000:00000000       ___safe_se_handler_count   00000000     <absolute>
 0000:00000000       ___safe_se_handler_table   00000000     <absolute>
 0001:0000001c       ??_C@_1BI@BHLBGEOK@?$AAP?$AAr?$AAi?$AAo?$AAr?$AAi?$AAt?$AAy?$AA2?$AA5?$AA6?$AA?$AA@ 1000101c     mddpcie950:mddpcie950.obj
 0001:00000034       ??_C@_1CC@KMPFMANC@?$AAD?$AAe?$AAv?$AAi?$AAc?$AAe?$AAA?$AAr?$AAr?$AAa?$AAy?$AAI?$AAn?$AAd?$AAe?$AAx?$AA?$AA@ 10001034     mddpcie950:mddpcie950.obj
 0001:000000d4       ??_C@_17KACEIPNC@?$AAK?$AAe?$AAy?$AA?$AA@ 100010d4     serpcie950:serpcie950.obj
 0001:000000e0       ??_7CSerialPDD@@6B@        100010e0     serpcie950:serpcie950.obj
 0001:000001d4       ??_C@_1CC@EKOCNIBB@?$AAC?$AAr?$AAy?$AAs?$AAt?$AAa?$AAl?$AAF?$AAr?$AAe?$AAq?$AAu?$AAe?$AAn?$AAc?$AAy?$AA?$AA@ 100011d4     serpcie950:serpcie950.obj
 0001:000001f8       ??_7CMiniThread@@6B@       100011f8     serpcie950:serpcie950.obj
 0001:000001fc       ??_7CSerialPDDPowerUpCallback@@6B@ 100011fc     serpcie950:serpcie950.obj
 0001:00000200       ??_7CRegpcie950@@6B@       10001200     pddpcie950:pddpcie950.obj
 0001:00000318       ??_C@_1CM@HIMBKDJM@?$AAL?$AAi?$AAn?$AAe?$AAD?$AAr?$AAi?$AAv?$AAe?$AAr?$AAD?$AAe?$AAl?$AAa?$AAy?$AAP?$AAh?$AAa?$AAs?$AAe@ 10001318     pddpcie950:pddpcie950.obj
 0001:00000344       ??_C@_1CI@GLAIJPLJ@?$AAL?$AAi?$AAn?$AAe?$AAD?$AAr?$AAi?$AAv?$AAe?$AAr?$AAD?$AAe?$AAl?$AAa?$AAy?$AAB?$AAi?$AAt?$AAs?$AA?$AA@ 10001344     pddpcie950:pddpcie950.obj
 0001:0000036c       ??_C@_1CE@PJBMNJAF@?$AAL?$AAi?$AAn?$AAe?$AAD?$AAr?$AAi?$AAv?$AAe?$AAr?$AAC?$AAo?$AAn?$AAt?$AAr?$AAo?$AAl?$AA?$AA@ 1000136c     pddpcie950:pddpcie950.obj
 0001:00000390       ??_C@_1CE@BHEKDMEI@?$AAB?$AAa?$AAu?$AAd?$AAr?$AAa?$AAt?$AAe?$AAM?$AAa?$AAp?$AAL?$AAi?$AAs?$AAt?$AAT?$AAo?$AA?$AA@ 10001390     pddpcie950:pddpcie950.obj
 0001:000003b4       ??_C@_1CI@OJPKJBA@?$AAB?$AAa?$AAu?$AAd?$AAr?$AAa?$AAt?$AAe?$AAM?$AAa?$AAp?$AAL?$AAi?$AAs?$AAt?$AAF?$AAr?$AAo?$AAm?$AA?$AA@ 100013b4     pddpcie950:pddpcie950.obj
 0001:000003dc       ??_C@_1CE@HLGCKFJ@?$AAF?$AAl?$AAo?$AAw?$AAC?$AAt?$AAr?$AAl?$AAH?$AAi?$AAg?$AAh?$AAL?$AAe?$AAv?$AAe?$AAl?$AA?$AA@ 100013dc     pddpcie950:pddpcie950.obj
 0001:00000400       ??_C@_1CC@ELLFOF@?$AAF?$AAl?$AAo?$AAw?$AAC?$AAt?$AAr?$AAl?$AAL?$AAo?$AAw?$AAL?$AAe?$AAv?$AAe?$AAl?$AA?$AA@ 10001400     pddpcie950:pddpcie950.obj
 0001:00000424       ??_C@_1BO@MCGADMLE@?$AAR?$AAx?$AAI?$AAn?$AAt?$AAT?$AAr?$AAi?$AAg?$AAL?$AAe?$AAv?$AAe?$AAl?$AA?$AA@ 10001424     pddpcie950:pddpcie950.obj
 0001:00000444       ??_C@_1BO@ELCCHGIE@?$AAT?$AAx?$AAI?$AAn?$AAt?$AAT?$AAr?$AAi?$AAg?$AAL?$AAe?$AAv?$AAe?$AAl?$AA?$AA@ 10001444     pddpcie950:pddpcie950.obj
 0001:00000464       ??_C@_1BA@BDHDGOBO@?$AAS?$AAy?$AAs?$AAI?$AAn?$AAt?$AAr?$AA?$AA@ 10001464     pddpcie950:pddpcie950.obj
 0001:00000474       ??_C@_1BE@PGPADFAN@?$AAR?$AAe?$AAg?$AAS?$AAt?$AAr?$AAi?$AAd?$AAe?$AA?$AA@ 10001474     pddpcie950:pddpcie950.obj
 0001:00000488       ??_C@_1BC@NIOILLNH@?$AAI?$AAN?$AAS?$AAT?$AAA?$AAN?$AAC?$AAE?$AA?$AA@ 10001488     pddpcie950:pddpcie950.obj
 0001:0000049c       ??_C@_17DBKELHOO@?$AAP?$AAN?$AAP?$AA?$AA@ 1000149c     pddpcie950:pddpcie950.obj
 0001:000004a4       ??_C@_1BC@DEOLOKPA@?$AA?2?$AAo?$AAp?$AAt?$AAi?$AAo?$AAn?$AA1?$AA?$AA@ 100014a4     pddpcie950:pddpcie950.obj
 0001:000004b8       ??_C@_1BI@FDNCMLGC@?$AAB?$AAU?$AAI?$AAL?$AAT?$AAI?$AAN?$AA?2?$AAP?$AAC?$AAI?$AA?$AA@ 100014b8     pddpcie950:pddpcie950.obj
 0001:000004d0       ??_7CMemRegpcie950@@6B@    100014d0     pddpcie950:pddpcie950.obj
 0001:00000608       ??_7CPddpcie950@@6BCSerialPDD@@@ 10001608     pddpcie950:pddpcie950.obj
 0001:0000070c       ??_7CPddpcie950@@6BCMiniThread@@@ 1000170c     pddpcie950:pddpcie950.obj
 0001:00000710       ??_7CPddpcie950Isr@@6BCSerialPDD@@@ 10001710     pddpcie950:pddisrpcie950.obj
 0001:00000814       ??_7CPddpcie950Isr@@6BCMiniThread@@@ 10001814     pddpcie950:pddisrpcie950.obj
 0001:00000818       ??_C@_1BE@GPBAGNPC@?$AAI?$AAs?$AAr?$AAH?$AAa?$AAn?$AAd?$AAl?$AAe?$AA?$AA@ 10001818     pddpcie950:pddisrpcie950.obj
 0001:00000830       ??_C@_1FM@FBAGINAI@?$AAF?$AAa?$AAi?$AAl?$AAe?$AAd?$AA?5?$AAt?$AAo?$AA?5?$AAg?$AAe?$AAt?$AA?5?$AAl?$AAo?$AAg?$AAi?$AAc?$AAa@ 10001830     pddpcie950:pddisrpcie950.obj
 0001:00000890       ??_C@_1FG@FPMLONNB@?$AAM?$AAe?$AAm?$AAo?$AAr?$AAy?$AA?5?$AAa?$AAl?$AAl?$AAo?$AAc?$AAa?$AAt?$AAi?$AAo?$AAn?$AA?5?$AAf?$AAa@ 10001890     pddpcie950:pddisrpcie950.obj
 0001:000008e8       ??_C@_1CA@INOAHGHF@?$AAB?$AAu?$AAs?$AAA?$AAc?$AAc?$AAe?$AAs?$AAs?$AAH?$AAa?$AAn?$AAd?$AAl?$AAe?$AA?$AA@ 100018e8     pddpcie950:pddisrpcie950.obj
 0001:00000908       ??_C@_1BC@MCDIKBIL@?$AAI?$AAs?$AAt?$AAE?$AAv?$AAe?$AAn?$AAt?$AA?$AA@ 10001908     pddpcie950:pddisrpcie950.obj
 0001:0000091c       ??_C@_1BG@LJAMCNJN@?$AAP?$AAo?$AAr?$AAt?$AAN?$AAu?$AAm?$AAb?$AAe?$AAr?$AA?$AA@ 1000191c     pddpcie950:pddisrpcie950.obj
 0001:00000994       ?CreateSerialObject@@YAPAVCSerialPDD@@PAGPAXPAU__HWOBJ@@K@Z 10001994 f   compcie950.obj
 0001:00000a9c       ?DeleteSerialObject@@YAXPAVCSerialPDD@@@Z 10001a9c f   compcie950.obj
 0001:00000ac0       DllEntry                   10001ac0 f   mddpcie950:mddpcie950.obj
 0001:00000ad8       DoTxData                   10001ad8 f   mddpcie950:mddpcie950.obj
 0001:00000c1c       DoRxData                   10001c1c f   mddpcie950:mddpcie950.obj
 0001:00000cf4       StopDispatchThread         10001cf4 f   mddpcie950:mddpcie950.obj
 0001:00000d88       ApplyDCB                   10001d88 f   mddpcie950:mddpcie950.obj
 0001:00000e04       COM_PreClose               10001e04 f   mddpcie950:mddpcie950.obj
 0001:00000ebc       PreClose                   10001ebc f   mddpcie950:mddpcie950.obj
 0001:00000ecc       COM_Close                  10001ecc f   mddpcie950:mddpcie950.obj
 0001:00000ff8       ProcessExiting             10001ff8 f   mddpcie950:mddpcie950.obj
 0001:0000102c       Close                      1000202c f   mddpcie950:mddpcie950.obj
 0001:0000103c       COM_PreDeinit              1000203c f   mddpcie950:mddpcie950.obj
 0001:000010a4       PreDeinit                  100020a4 f   mddpcie950:mddpcie950.obj
 0001:000010b4       COM_Deinit                 100020b4 f   mddpcie950:mddpcie950.obj
 0001:000011d8       Deinit                     100021d8 f   mddpcie950:mddpcie950.obj
 0001:000011e8       COM_Read                   100021e8 f   mddpcie950:mddpcie950.obj
 0001:0000144c       Read                       1000244c f   mddpcie950:mddpcie950.obj
 0001:0000145c       COM_Seek                   1000245c f   mddpcie950:mddpcie950.obj
 0001:00001464       Seek                       10002464 f   mddpcie950:mddpcie950.obj
 0001:0000146c       COM_PowerUp                1000246c f   mddpcie950:mddpcie950.obj
 0001:000014ac       PowerUp                    100024ac f   mddpcie950:mddpcie950.obj
 0001:000014bc       COM_PowerDown              100024bc f   mddpcie950:mddpcie950.obj
 0001:000014fc       PowerDown                  100024fc f   mddpcie950:mddpcie950.obj
 0001:0000150c       WaitCommEvent              1000250c f   mddpcie950:mddpcie950.obj
 0001:0000161c       EvaluateEventFlag          1000261c f   mddpcie950:mddpcie950.obj
 0001:000016bc       COM_IOControl              100026bc f   mddpcie950:mddpcie950.obj
 0001:00002150       IOControl                  10003150 f   mddpcie950:mddpcie950.obj
 0001:00002180       SerialEventHandler         10003180 f   mddpcie950:mddpcie950.obj
 0001:000022f4       StartDispatchThread        100032f4 f   mddpcie950:mddpcie950.obj
 0001:00002384       COM_Init                   10003384 f   mddpcie950:mddpcie950.obj
 0001:0000261c       Init                       1000361c f   mddpcie950:mddpcie950.obj
 0001:0000262c       COM_Open                   1000362c f   mddpcie950:mddpcie950.obj
 0001:000028c4       Open                       100038c4 f   mddpcie950:mddpcie950.obj
 0001:000028d4       COM_Write                  100038d4 f   mddpcie950:mddpcie950.obj
 0001:00002a34       Write                      10003a34 f   mddpcie950:mddpcie950.obj
 0001:00002a44       ?GetRegValue@CRegistryEdit@@QAAHPBGPAEK@Z 10003a44 f i serpcie950:serpcie950.obj
 0001:00002a94       ?ThreadStart@CMiniThread@@QAAHXZ 10003a94 f i serpcie950:serpcie950.obj
 0001:00002ad4       ?WaitThreadComplete@CMiniThread@@QAAHK@Z 10003ad4 f i serpcie950:serpcie950.obj
 0001:00002b34       ?ForceTerminated@CMiniThread@@QAAHXZ 10003b34 f i serpcie950:serpcie950.obj
 0001:00002b84       ?ThreadProc@CMiniThread@@CAKPAX@Z 10003b84 f i serpcie950:serpcie950.obj
 0001:00002bb4       ?ThreadRun@CSerialPDDPowerUpCallback@@EAAKXZ 10003bb4 f   serpcie950:serpcie950.obj
 0001:00002c24       ??0CSerialPDD@@QAA@PAGPAXPAU__HWOBJ@@@Z 10003c24 f   serpcie950:serpcie950.obj
 0001:00002d28       ?GetDevicePowerState@CSerialPDD@@UAA?AW4_CEDEVICE_POWER_STATE@@XZ 10003d28 f i serpcie950:serpcie950.obj
 0001:00002d30       ?GetPowerCapabilities@CSerialPDD@@UAA?AU_POWER_CAPABILITIES@@XZ 10003d30 f i serpcie950:serpcie950.obj
 0001:00002d54       ?IsCTSOff@CSerialPDD@@UAAHXZ 10003d54 f i serpcie950:serpcie950.obj
 0001:00002d80       ?IsDSROff@CSerialPDD@@UAAHXZ 10003d80 f i serpcie950:serpcie950.obj
 0001:00002dac       ?SetFifoCtrlLevels@CSerialPDD@@UAAHPAUFIFO_LEVEL_CTRL_VALS@@@Z 10003dac f i serpcie950:serpcie950.obj
 0001:00002db4       ?SetInternalLoopback@CSerialPDD@@UAAXH@Z 10003db4 f i serpcie950:serpcie950.obj
 0001:00002db8       ?SaveBaudrateMap@CSerialPDD@@UAAHPAUBAUDRATE_MAP@@@Z 10003db8 f i serpcie950:serpcie950.obj
 0001:00002dc0       ?RegSetPnpValue@CSerialPDD@@UAAHPBGKPBEK@Z 10003dc0 f i serpcie950:serpcie950.obj
 0001:00002dc8       ?GetLineDriverControls@CSerialPDD@@UAAHPAULINE_DRIVER_CONTROL@@K@Z 10003dc8 f i serpcie950:serpcie950.obj
 0001:00002dd0       ?SetLineDriverControls@CSerialPDD@@UAAHPAULINE_DRIVER_CONTROL@@K@Z 10003dd0 f i serpcie950:serpcie950.obj
 0001:00002dd8       ?SaveLineDriverControls@CSerialPDD@@UAAHPAULINE_DRIVER_CONTROL@@@Z 10003dd8 f i serpcie950:serpcie950.obj
 0001:00002de0       ?SetOutputMode@CSerialPDD@@UAAXHH@Z 10003de0 f i serpcie950:serpcie950.obj
 0001:00002dec       ?GetOutputMode@CSerialPDD@@UAAXPAH0@Z 10003dec f i serpcie950:serpcie950.obj
 0001:00002e08       ?PostInit@CSerialPDD@@UAAXXZ 10003e08 f   serpcie950:serpcie950.obj
 0001:00002e44       ?Open@CSerialPDD@@UAAHXZ   10003e44 f   serpcie950:serpcie950.obj
 0001:00002ee4       ?Close@CSerialPDD@@UAAHXZ  10003ee4 f   serpcie950:serpcie950.obj
 0001:00002f84       ?Reset@CSerialPDD@@QAAXXZ  10003f84 f   serpcie950:serpcie950.obj
 0001:00003020       ?Ioctl@CSerialPDD@@UAAHKPAEK0KPAK@Z 10004020 f   serpcie950:serpcie950.obj
 0001:00003470       ?InitialPower@CSerialPDD@@UAAHH@Z 10004470 f   serpcie950:serpcie950.obj
 0001:0000348c       ?SetPowerStateStatic@CSerialPDD@@KA?AW4_CEDEVICE_POWER_STATE@@KW42@@Z 1000448c f   serpcie950:serpcie950.obj
 0001:00003508       ?PowerOff@CSerialPDD@@UAAHXZ 10004508 f   serpcie950:serpcie950.obj
 0001:00003550       ?PowerOn@CSerialPDD@@UAAHXZ 10004550 f   serpcie950:serpcie950.obj
 0001:000035c0       ?SetDevicePowerState@CSerialPDD@@UAAHW4_CEDEVICE_POWER_STATE@@@Z 100045c0 f   serpcie950:serpcie950.obj
 0001:00003690       ?InitialEnableInterrupt@CSerialPDD@@UAAHH@Z 10004690 f   serpcie950:serpcie950.obj
 0001:000036bc       ?NotifyPDDInterrupt@CSerialPDD@@UAAHW4INTERRUPT_TYPE@@@Z 100046bc f   serpcie950:serpcie950.obj
 0001:00003754       ?GetInterruptType@CSerialPDD@@UAA?AW4INTERRUPT_TYPE@@XZ 10004754 f   serpcie950:serpcie950.obj
 0001:00003784       ?DataReplaced@CSerialPDD@@UAAHPAEH@Z 10004784 f   serpcie950:serpcie950.obj
 0001:00003820       ?EventCallback@CSerialPDD@@UAAHKK@Z 10004820 f   serpcie950:serpcie950.obj
 0001:00003864       ?PurgeComm@CSerialPDD@@UAAHK@Z 10004864 f   serpcie950:serpcie950.obj
 0001:000038a8       ?SetReceiveError@CSerialPDD@@UAAXK@Z 100048a8 f   serpcie950:serpcie950.obj
 0001:000038f8       ?GetReceivedError@CSerialPDD@@UAAKXZ 100048f8 f   serpcie950:serpcie950.obj
 0001:00003928       ?SetDefaultConfiguration@CSerialPDD@@UAAXXZ 10004928 f   serpcie950:serpcie950.obj
 0001:00003a48       ?SetDCB@CSerialPDD@@UAAHPAU_DCB@@@Z 10004a48 f   serpcie950:serpcie950.obj
 0001:00003bdc       ?SerInit@@YAPAXKPAXPAU__HWOBJ@@@Z 10004bdc f   serpcie950:serpcie950.obj
 0001:00003c1c       ?SerDeinit@@YAKPAX@Z       10004c1c f   serpcie950:serpcie950.obj
 0001:00003c58       ?SerPostInit@@YAHPAX@Z     10004c58 f   serpcie950:serpcie950.obj
 0001:00003c7c       ?SerOpen@@YAHPAX@Z         10004c7c f   serpcie950:serpcie950.obj
 0001:00003ca4       ?SerClose@@YAKPAX@Z        10004ca4 f   serpcie950:serpcie950.obj
 0001:00003ccc       ?SerGetInterruptType@@YA?AW4INTERRUPT_TYPE@@PAX@Z 10004ccc f   serpcie950:serpcie950.obj
 0001:00003cf4       ?SerRxIntr@@YAKPAXPAEPAK@Z 10004cf4 f   serpcie950:serpcie950.obj
 0001:00003d1c       ?SerTxIntrEx@@YAXPAXPAEPAK@Z 10004d1c f   serpcie950:serpcie950.obj
 0001:00003d3c       ?SerModemIntr@@YAXPAX@Z    10004d3c f   serpcie950:serpcie950.obj
 0001:00003d78       ?SerLineIntr@@YAXPAX@Z     10004d78 f   serpcie950:serpcie950.obj
 0001:00003db4       ?SerGetRxBufferSize@@YAKPAX@Z 10004db4 f   serpcie950:serpcie950.obj
 0001:00003df8       ?SerPowerOff@@YAHPAX@Z     10004df8 f   serpcie950:serpcie950.obj
 0001:00003e3c       ?SerPowerOn@@YAHPAX@Z      10004e3c f   serpcie950:serpcie950.obj
 0001:00003e80       ?SerClearDTR@@YAXPAX@Z     10004e80 f   serpcie950:serpcie950.obj
 0001:00003ec0       ?SerSetDTR@@YAXPAX@Z       10004ec0 f   serpcie950:serpcie950.obj
 0001:00003f00       ?SerClearRTS@@YAXPAX@Z     10004f00 f   serpcie950:serpcie950.obj
 0001:00003f40       ?SerSetRTS@@YAXPAX@Z       10004f40 f   serpcie950:serpcie950.obj
 0001:00003f80       ?SerEnableIR@@YAHPAXK@Z    10004f80 f   serpcie950:serpcie950.obj
 0001:00003fd4       ?SerDisableIR@@YAHPAX@Z    10004fd4 f   serpcie950:serpcie950.obj
 0001:00004000       ?SerClearBreak@@YAXPAX@Z   10005000 f   serpcie950:serpcie950.obj
 0001:00004040       ?SerSetBreak@@YAXPAX@Z     10005040 f   serpcie950:serpcie950.obj
 0001:00004080       ?SerXmitComChar@@YAHPAXE@Z 10005080 f   serpcie950:serpcie950.obj
 0001:000040c0       ?SerGetStatus@@YAKPAXPAU_COMSTAT@@@Z 100050c0 f   serpcie950:serpcie950.obj
 0001:000041e8       ?SerReset@@YAXPAX@Z        100051e8 f   serpcie950:serpcie950.obj
 0001:000041fc       ?SerGetModemStatus@@YAXPAXPAK@Z 100051fc f   serpcie950:serpcie950.obj
 0001:00004248       ?SerGetCommProperties@@YAXPAXPAU_COMMPROP@@@Z 10005248 f   serpcie950:serpcie950.obj
 0001:00004270       ?SerPurgeComm@@YAXPAXK@Z   10005270 f   serpcie950:serpcie950.obj
 0001:000042ac       ?SerSetDCB@@YAHPAXPAU_DCB@@@Z 100052ac f   serpcie950:serpcie950.obj
 0001:000042f8       ?SerSetCommTimeouts@@YAHPAXPAU_COMMTIMEOUTS@@@Z 100052f8 f   serpcie950:serpcie950.obj
 0001:00004300       ?SerEnableXmit@@YAXPAXH@Z  10005300 f   serpcie950:serpcie950.obj
 0001:0000433c       ?SerIoctl@@YAHPAXKPAEK1KPAK@Z 1000533c f   serpcie950:serpcie950.obj
 0001:000043a0       GetSerialObject            100053a0 f   serpcie950:serpcie950.obj
 0001:000043dc       ??0CMiniThread@@QAA@KH@Z   100053dc f i serpcie950:serpcie950.obj
 0001:00004448       ??0CSerialPDDPowerUpCallback@@QAA@PAVCSerialPDD@@@Z 10005448 f   serpcie950:serpcie950.obj
 0001:000044a0       ??1CSerialPDDPowerUpCallback@@QAA@XZ 100054a0 f   serpcie950:serpcie950.obj
 0001:000044fc       ?Init@CSerialPDD@@UAAHXZ   100054fc f   serpcie950:serpcie950.obj
 0001:000045b4       ??1CSerialPDD@@UAA@XZ      100055b4 f   serpcie950:serpcie950.obj
 0001:00004654       ??_ECSerialPDD@@UAAPAXI@Z  10005654 f i serpcie950:serpcie950.obj
 0001:00004654       ??_GCSerialPDD@@UAAPAXI@Z  10005654 f i serpcie950:serpcie950.obj
 0001:0000467c       ??0CRegistryEdit@@QAA@PAUHKEY__@@PBG@Z 1000567c f i pddpcie950:pddpcie950.obj
 0001:000046cc       ?Init@CRegpcie950@@UAAHXZ  100056cc f i pddpcie950:pddpcie950.obj
 0001:000046e0       ?Write_DATA@CRegpcie950@@UAAXE@Z 100056e0 f i pddpcie950:pddpcie950.obj
 0001:000046f4       ?Read_Data@CRegpcie950@@UAAEXZ 100056f4 f i pddpcie950:pddpcie950.obj
 0001:00004708       ?Write_IER@CRegpcie950@@UAAXE@Z 10005708 f i pddpcie950:pddpcie950.obj
 0001:0000471c       ?Read_IER@CRegpcie950@@UAAEXZ 1000571c f i pddpcie950:pddpcie950.obj
 0001:00004730       ?Write_FCR@CRegpcie950@@UAAXE@Z 10005730 f i pddpcie950:pddpcie950.obj
 0001:00004754       ?Read_FCR@CRegpcie950@@UAAEXZ 10005754 f i pddpcie950:pddpcie950.obj
 0001:0000475c       ?Read_IIR@CRegpcie950@@UAAEXZ 1000575c f i pddpcie950:pddpcie950.obj
 0001:00004770       ?Write_LCR@CRegpcie950@@UAAXE@Z 10005770 f i pddpcie950:pddpcie950.obj
 0001:00004784       ?Read_LCR@CRegpcie950@@UAAEXZ 10005784 f i pddpcie950:pddpcie950.obj
 0001:00004798       ?Write_MCR@CRegpcie950@@UAAXE@Z 10005798 f i pddpcie950:pddpcie950.obj
 0001:000047ac       ?Read_MCR@CRegpcie950@@UAAEXZ 100057ac f i pddpcie950:pddpcie950.obj
 0001:000047c0       ?Write_LSR@CRegpcie950@@UAAXE@Z 100057c0 f i pddpcie950:pddpcie950.obj
 0001:000047d4       ?Read_LSR@CRegpcie950@@UAAEXZ 100057d4 f i pddpcie950:pddpcie950.obj
 0001:000047e8       ?Write_MSR@CRegpcie950@@UAAXE@Z 100057e8 f i pddpcie950:pddpcie950.obj
 0001:000047fc       ?Read_MSR@CRegpcie950@@UAAEXZ 100057fc f i pddpcie950:pddpcie950.obj
 0001:00004810       ?Write_SPR@CRegpcie950@@UAAXE@Z 10005810 f i pddpcie950:pddpcie950.obj
 0001:00004824       ?Read_SPR@CRegpcie950@@UAAEXZ 10005824 f i pddpcie950:pddpcie950.obj
 0001:00004838       ?Write_DIVISOR@CRegpcie950@@UAAXG@Z 10005838 f i pddpcie950:pddpcie950.obj
 0001:00004884       ?Read_DIVISOR@CRegpcie950@@UAAGXZ 10005884 f i pddpcie950:pddpcie950.obj
 0001:000048d0       ?Write_EFR@CRegpcie950@@UAAXE@Z 100058d0 f i pddpcie950:pddpcie950.obj
 0001:000048f4       ?Read_EFR@CRegpcie950@@UAAEXZ 100058f4 f i pddpcie950:pddpcie950.obj
 0001:00004914       ?Write_XON1@CRegpcie950@@UAAXE@Z 10005914 f i pddpcie950:pddpcie950.obj
 0001:00004938       ?Read_XON1@CRegpcie950@@UAAEXZ 10005938 f i pddpcie950:pddpcie950.obj
 0001:00004958       ?Write_XON2@CRegpcie950@@UAAXE@Z 10005958 f i pddpcie950:pddpcie950.obj
 0001:0000497c       ?Read_XON2@CRegpcie950@@UAAEXZ 1000597c f i pddpcie950:pddpcie950.obj
 0001:0000499c       ?Write_XOFF1@CRegpcie950@@UAAXE@Z 1000599c f i pddpcie950:pddpcie950.obj
 0001:000049c0       ?Read_XOFF1@CRegpcie950@@UAAEXZ 100059c0 f i pddpcie950:pddpcie950.obj
 0001:000049e0       ?Write_XOFF2@CRegpcie950@@UAAXE@Z 100059e0 f i pddpcie950:pddpcie950.obj
 0001:00004a04       ?Read_XOFF2@CRegpcie950@@UAAEXZ 10005a04 f i pddpcie950:pddpcie950.obj
 0001:00004a24       ?Write_ASR@CRegpcie950@@UAAXE@Z 10005a24 f i pddpcie950:pddpcie950.obj
 0001:00004a48       ?Read_ASR@CRegpcie950@@UAAEXZ 10005a48 f i pddpcie950:pddpcie950.obj
 0001:00004a68       ?Read_RFL@CRegpcie950@@UAAEXZ 10005a68 f i pddpcie950:pddpcie950.obj
 0001:00004ad8       ?Read_TFL@CRegpcie950@@UAAEXZ 10005ad8 f i pddpcie950:pddpcie950.obj
 0001:00004b48       ?Write_ACR@CRegpcie950@@UAAXE@Z 10005b48 f i pddpcie950:pddpcie950.obj
 0001:00004b6c       ?Read_ACR@CRegpcie950@@UAAEXZ 10005b6c f i pddpcie950:pddpcie950.obj
 0001:00004b8c       ?Write_CPR@CRegpcie950@@UAAXE@Z 10005b8c f i pddpcie950:pddpcie950.obj
 0001:00004bb0       ?Read_CPR@CRegpcie950@@UAAEXZ 10005bb0 f i pddpcie950:pddpcie950.obj
 0001:00004bd0       ?Write_TCR@CRegpcie950@@UAAXE@Z 10005bd0 f i pddpcie950:pddpcie950.obj
 0001:00004bf4       ?Read_TCR@CRegpcie950@@UAAEXZ 10005bf4 f i pddpcie950:pddpcie950.obj
 0001:00004c14       ?Write_TTL@CRegpcie950@@UAAXE@Z 10005c14 f i pddpcie950:pddpcie950.obj
 0001:00004c38       ?Read_TTL@CRegpcie950@@UAAEXZ 10005c38 f i pddpcie950:pddpcie950.obj
 0001:00004c58       ?Write_RTL@CRegpcie950@@UAAXE@Z 10005c58 f i pddpcie950:pddpcie950.obj
 0001:00004c7c       ?Read_RTL@CRegpcie950@@UAAEXZ 10005c7c f i pddpcie950:pddpcie950.obj
 0001:00004c9c       ?Write_FCL@CRegpcie950@@UAAXE@Z 10005c9c f i pddpcie950:pddpcie950.obj
 0001:00004cc0       ?Read_FCL@CRegpcie950@@UAAEXZ 10005cc0 f i pddpcie950:pddpcie950.obj
 0001:00004ce0       ?Write_FCH@CRegpcie950@@UAAXE@Z 10005ce0 f i pddpcie950:pddpcie950.obj
 0001:00004d04       ?Read_FCH@CRegpcie950@@UAAEXZ 10005d04 f i pddpcie950:pddpcie950.obj
 0001:00004d24       ?Write_NMR@CRegpcie950@@UAAXE@Z 10005d24 f i pddpcie950:pddpcie950.obj
 0001:00004d48       ?Read_NMR@CRegpcie950@@UAAEXZ 10005d48 f i pddpcie950:pddpcie950.obj
 0001:00004d68       ?Write_MDM@CRegpcie950@@UAAXE@Z 10005d68 f i pddpcie950:pddpcie950.obj
 0001:00004d8c       ?Read_MDM@CRegpcie950@@UAAEXZ 10005d8c f i pddpcie950:pddpcie950.obj
 0001:00004dac       ?Write_485CR@CRegpcie950@@UAAXE@Z 10005dac f i pddpcie950:pddpcie950.obj
 0001:00004dd0       ?Read_485CR@CRegpcie950@@UAAEXZ 10005dd0 f i pddpcie950:pddpcie950.obj
 0001:00004df0       ?Write_485DR@CRegpcie950@@UAAXE@Z 10005df0 f i pddpcie950:pddpcie950.obj
 0001:00004e14       ?Read_485DR@CRegpcie950@@UAAEXZ 10005e14 f i pddpcie950:pddpcie950.obj
 0001:00004e34       ?Read_ID1@CRegpcie950@@UAAEXZ 10005e34 f i pddpcie950:pddpcie950.obj
 0001:00004e54       ?Read_ID2@CRegpcie950@@UAAEXZ 10005e54 f i pddpcie950:pddpcie950.obj
 0001:00004e74       ?Read_ID3@CRegpcie950@@UAAEXZ 10005e74 f i pddpcie950:pddpcie950.obj
 0001:00004e94       ?WRITE_550_PORT@CRegpcie950@@UAAXPAEE@Z 10005e94 f i pddpcie950:pddpcie950.obj
 0001:00004edc       ?READ_550_PORT@CRegpcie950@@UAAEPAE@Z 10005edc f i pddpcie950:pddpcie950.obj
 0001:00004f24       ?WRITE_650_PORT@CRegpcie950@@UAAXPAEE@Z 10005f24 f i pddpcie950:pddpcie950.obj
 0001:00004f3c       ?READ_650_PORT@CRegpcie950@@UAAEPAE@Z 10005f3c f i pddpcie950:pddpcie950.obj
 0001:00004f50       ?WRITE_950_PORT@CRegpcie950@@UAAXPAEE@Z 10005f50 f i pddpcie950:pddpcie950.obj
 0001:00004f68       ?READ_950_PORT@CRegpcie950@@UAAEPAE@Z 10005f68 f i pddpcie950:pddpcie950.obj
 0001:00004f7c       ?WRITE_ICR_PORT@CRegpcie950@@UAAXPAEE@Z 10005f7c f i pddpcie950:pddpcie950.obj
 0001:00004f94       ?READ_ICR_PORT@CRegpcie950@@UAAEPAE@Z 10005f94 f i pddpcie950:pddpcie950.obj
 0001:00004fa8       ??_GCRegpcie950@@UAAPAXI@Z 10005fa8 f i pddpcie950:pddpcie950.obj
 0001:00004fa8       ??_ECRegpcie950@@UAAPAXI@Z 10005fa8 f i pddpcie950:pddpcie950.obj
 0001:00004fdc       ??0CRegpcie950@@QAA@PAEK@Z 10005fdc f   pddpcie950:pddpcie950.obj
 0001:000051a4       ?Backup@CRegpcie950@@UAAXXZ 100061a4 f   pddpcie950:pddpcie950.obj
 0001:000053fc       ?Restore@CRegpcie950@@UAAXXZ 100063fc f   pddpcie950:pddpcie950.obj
 0001:000055fc       ?Init@CPddpcie950@@UAAHXZ  100065fc f   pddpcie950:pddpcie950.obj
 0001:00005938       ?GetRegMultiDword@CPddpcie950@@EAAHPBGPAKK@Z 10006938 f   pddpcie950:pddpcie950.obj
 0001:000059d0       ?MapHardware@CPddpcie950@@UAAHXZ 100069d0 f   pddpcie950:pddpcie950.obj
 0001:00005b60       ?PostInit@CPddpcie950@@UAAXXZ 10006b60 f   pddpcie950:pddpcie950.obj
 0001:00005cb4       ?ThreadRun@CPddpcie950@@EAAKXZ 10006cb4 f   pddpcie950:pddpcie950.obj
 0001:00005e14       ?InitialEnableInterrupt@CPddpcie950@@UAAHH@Z 10006e14 f   pddpcie950:pddpcie950.obj
 0001:00005f04       ?InitXmit@CPddpcie950@@UAAHH@Z 10006f04 f   pddpcie950:pddpcie950.obj
 0001:00005f88       ?GetWriteableSize@CPddpcie950@@UAAKXZ 10006f88 f   pddpcie950:pddpcie950.obj
 0001:00005fac       ?PushPriorityFifo@CPddpcie950@@IAAXE@Z 10006fac f   pddpcie950:pddpcie950.obj
 0001:00006040       ?PopPriorityFifo@CPddpcie950@@IAAHPAE@Z 10007040 f   pddpcie950:pddpcie950.obj
 0001:000060a8       ?XmitComChar@CPddpcie950@@UAAXE@Z 100070a8 f   pddpcie950:pddpcie950.obj
 0001:0000611c       ?EnableReceiveInterrupt@CPddpcie950@@UAAHH@Z 1000711c f   pddpcie950:pddpcie950.obj
 0001:000061bc       ?EnableXmitInterrupt@CPddpcie950@@UAAHH@Z 100071bc f   pddpcie950:pddpcie950.obj
 0001:0000625c       ?CancelXmit@CPddpcie950@@UAAHXZ 1000725c f   pddpcie950:pddpcie950.obj
 0001:000062b0       ?EmptyEventData@CPddpcie950@@UAAXXZ 100072b0 f   pddpcie950:pddpcie950.obj
 0001:000062b4       ?InitReceive@CPddpcie950@@UAAHH@Z 100072b4 f   pddpcie950:pddpcie950.obj
 0001:00006384       ?GetReadableSize@CPddpcie950@@IAAKXZ 10007384 f   pddpcie950:pddpcie950.obj
 0001:000063c0       ?ReceiveInterruptHandler@CPddpcie950@@UAAKPAEPAK@Z 100073c0 f   pddpcie950:pddpcie950.obj
 0001:000064a8       ?CancelReceive@CPddpcie950@@UAAKXZ 100074a8 f   pddpcie950:pddpcie950.obj
 0001:00006504       ?InitModem@CPddpcie950@@UAAHH@Z 10007504 f   pddpcie950:pddpcie950.obj
 0001:0000658c       ?GetModemStatus@CPddpcie950@@UAAKXZ 1000758c f   pddpcie950:pddpcie950.obj
 0001:0000661c       ?SetDTR@CPddpcie950@@UAAXH@Z 1000761c f   pddpcie950:pddpcie950.obj
 0001:00006674       ?SetRTS@CPddpcie950@@UAAXH@Z 10007674 f   pddpcie950:pddpcie950.obj
 0001:000066cc       ?InitLine@CPddpcie950@@UAAHH@Z 100076cc f   pddpcie950:pddpcie950.obj
 0001:0000676c       ?GetLineStatus@CPddpcie950@@QAAEXZ 1000776c f   pddpcie950:pddpcie950.obj
 0001:000067ec       ?SetBreak@CPddpcie950@@UAAXH@Z 100077ec f   pddpcie950:pddpcie950.obj
 0001:00006844       ?GetBaudConfigFromBaudRate@CPddpcie950@@IAAHKJPAU_BAUD_CONFIG@1@@Z 10007844 f   pddpcie950:pddpcie950.obj
 0001:000069ac       ?SetBaudRate@CPddpcie950@@UAAHKH@Z 100079ac f   pddpcie950:pddpcie950.obj
 0001:00006a84       ?SetByteSize@CPddpcie950@@UAAHK@Z 10007a84 f   pddpcie950:pddpcie950.obj
 0001:00006b14       ?SetParity@CPddpcie950@@UAAHK@Z 10007b14 f   pddpcie950:pddpcie950.obj
 0001:00006ba4       ?SetStopBits@CPddpcie950@@UAAHK@Z 10007ba4 f   pddpcie950:pddpcie950.obj
 0001:00006c08       ?SetFlowControl@CPddpcie950@@UAAHPAU_DCB@@@Z 10007c08 f   pddpcie950:pddpcie950.obj
 0001:00006e8c       ?GetXonXoffStatus@CPddpcie950@@UAAXPAU_COMSTAT@@@Z 10007e8c f   pddpcie950:pddpcie950.obj
 0001:00006f38       ?EnableXmit@CPddpcie950@@UAAXH@Z 10007f38 f   pddpcie950:pddpcie950.obj
 0001:00006f80       ?SetFifoCtrlLevels@CPddpcie950@@UAAHPAUFIFO_LEVEL_CTRL_VALS@@@Z 10007f80 f   pddpcie950:pddpcie950.obj
 0001:0000714c       ?SetInternalLoopback@CPddpcie950@@UAAXH@Z 1000814c f   pddpcie950:pddpcie950.obj
 0001:000071b4       ?GetLineDriverControls@CPddpcie950@@UAAHPAULINE_DRIVER_CONTROL@@K@Z 100081b4 f   pddpcie950:pddpcie950.obj
 0001:00007280       ?SetLineDriverControls@CPddpcie950@@UAAHPAULINE_DRIVER_CONTROL@@K@Z 10008280 f   pddpcie950:pddpcie950.obj
 0001:00007378       ?SaveLineDriverControls@CPddpcie950@@UAAHPAULINE_DRIVER_CONTROL@@@Z 10008378 f   pddpcie950:pddpcie950.obj
 0001:0000742c       ?SaveBaudrateMap@CPddpcie950@@UAAHPAUBAUDRATE_MAP@@@Z 1000842c f   pddpcie950:pddpcie950.obj
 0001:00007640       ?RegSetPnpValue@CPddpcie950@@UAAHPBGKPBEK@Z 10008640 f   pddpcie950:pddpcie950.obj
 0001:0000778c       ?Write_DATA@CMemRegpcie950@@UAAXE@Z 1000878c f i pddpcie950:pddpcie950.obj
 0001:000077a0       ?Read_Data@CMemRegpcie950@@UAAEXZ 100087a0 f i pddpcie950:pddpcie950.obj
 0001:000077b4       ?Write_IER@CMemRegpcie950@@UAAXE@Z 100087b4 f i pddpcie950:pddpcie950.obj
 0001:000077c8       ?Read_IER@CMemRegpcie950@@UAAEXZ 100087c8 f i pddpcie950:pddpcie950.obj
 0001:000077dc       ?Write_FCR@CMemRegpcie950@@UAAXE@Z 100087dc f i pddpcie950:pddpcie950.obj
 0001:00007800       ?Read_IIR@CMemRegpcie950@@UAAEXZ 10008800 f i pddpcie950:pddpcie950.obj
 0001:00007814       ?Write_LCR@CMemRegpcie950@@UAAXE@Z 10008814 f i pddpcie950:pddpcie950.obj
 0001:00007828       ?Read_LCR@CMemRegpcie950@@UAAEXZ 10008828 f i pddpcie950:pddpcie950.obj
 0001:0000783c       ?Write_MCR@CMemRegpcie950@@UAAXE@Z 1000883c f i pddpcie950:pddpcie950.obj
 0001:00007850       ?Read_MCR@CMemRegpcie950@@UAAEXZ 10008850 f i pddpcie950:pddpcie950.obj
 0001:00007864       ?Write_LSR@CMemRegpcie950@@UAAXE@Z 10008864 f i pddpcie950:pddpcie950.obj
 0001:00007878       ?Read_LSR@CMemRegpcie950@@UAAEXZ 10008878 f i pddpcie950:pddpcie950.obj
 0001:0000788c       ?Write_MSR@CMemRegpcie950@@UAAXE@Z 1000888c f i pddpcie950:pddpcie950.obj
 0001:000078a0       ?Read_MSR@CMemRegpcie950@@UAAEXZ 100088a0 f i pddpcie950:pddpcie950.obj
 0001:000078b4       ?Write_SPR@CMemRegpcie950@@UAAXE@Z 100088b4 f i pddpcie950:pddpcie950.obj
 0001:000078c8       ?Read_SPR@CMemRegpcie950@@UAAEXZ 100088c8 f i pddpcie950:pddpcie950.obj
 0001:000078dc       ?Write_DIVISOR@CMemRegpcie950@@UAAXG@Z 100088dc f i pddpcie950:pddpcie950.obj
 0001:00007928       ?Read_DIVISOR@CMemRegpcie950@@UAAGXZ 10008928 f i pddpcie950:pddpcie950.obj
 0001:00007974       ?Write_EFR@CMemRegpcie950@@UAAXE@Z 10008974 f i pddpcie950:pddpcie950.obj
 0001:00007998       ?Read_EFR@CMemRegpcie950@@UAAEXZ 10008998 f i pddpcie950:pddpcie950.obj
 0001:000079b8       ?Write_XON1@CMemRegpcie950@@UAAXE@Z 100089b8 f i pddpcie950:pddpcie950.obj
 0001:000079dc       ?Read_XON1@CMemRegpcie950@@UAAEXZ 100089dc f i pddpcie950:pddpcie950.obj
 0001:000079fc       ?Write_XON2@CMemRegpcie950@@UAAXE@Z 100089fc f i pddpcie950:pddpcie950.obj
 0001:00007a20       ?Read_XON2@CMemRegpcie950@@UAAEXZ 10008a20 f i pddpcie950:pddpcie950.obj
 0001:00007a40       ?Write_XOFF1@CMemRegpcie950@@UAAXE@Z 10008a40 f i pddpcie950:pddpcie950.obj
 0001:00007a64       ?Read_XOFF1@CMemRegpcie950@@UAAEXZ 10008a64 f i pddpcie950:pddpcie950.obj
 0001:00007a84       ?Write_XOFF2@CMemRegpcie950@@UAAXE@Z 10008a84 f i pddpcie950:pddpcie950.obj
 0001:00007aa8       ?Read_XOFF2@CMemRegpcie950@@UAAEXZ 10008aa8 f i pddpcie950:pddpcie950.obj
 0001:00007ac8       ?Write_ASR@CMemRegpcie950@@UAAXE@Z 10008ac8 f i pddpcie950:pddpcie950.obj
 0001:00007aec       ?Read_ASR@CMemRegpcie950@@UAAEXZ 10008aec f i pddpcie950:pddpcie950.obj
 0001:00007b0c       ?Read_RFL@CMemRegpcie950@@UAAEXZ 10008b0c f i pddpcie950:pddpcie950.obj
 0001:00007b7c       ?Read_TFL@CMemRegpcie950@@UAAEXZ 10008b7c f i pddpcie950:pddpcie950.obj
 0001:00007bec       ?Write_ACR@CMemRegpcie950@@UAAXE@Z 10008bec f i pddpcie950:pddpcie950.obj
 0001:00007c10       ?Read_ACR@CMemRegpcie950@@UAAEXZ 10008c10 f i pddpcie950:pddpcie950.obj
 0001:00007c30       ?Write_CPR@CMemRegpcie950@@UAAXE@Z 10008c30 f i pddpcie950:pddpcie950.obj
 0001:00007c54       ?Read_CPR@CMemRegpcie950@@UAAEXZ 10008c54 f i pddpcie950:pddpcie950.obj
 0001:00007c74       ?Write_TCR@CMemRegpcie950@@UAAXE@Z 10008c74 f i pddpcie950:pddpcie950.obj
 0001:00007c98       ?Read_TCR@CMemRegpcie950@@UAAEXZ 10008c98 f i pddpcie950:pddpcie950.obj
 0001:00007cb8       ?Write_TTL@CMemRegpcie950@@UAAXE@Z 10008cb8 f i pddpcie950:pddpcie950.obj
 0001:00007cdc       ?Read_TTL@CMemRegpcie950@@UAAEXZ 10008cdc f i pddpcie950:pddpcie950.obj
 0001:00007cfc       ?Write_RTL@CMemRegpcie950@@UAAXE@Z 10008cfc f i pddpcie950:pddpcie950.obj
 0001:00007d20       ?Read_RTL@CMemRegpcie950@@UAAEXZ 10008d20 f i pddpcie950:pddpcie950.obj
 0001:00007d40       ?Write_FCL@CMemRegpcie950@@UAAXE@Z 10008d40 f i pddpcie950:pddpcie950.obj
 0001:00007d64       ?Read_FCL@CMemRegpcie950@@UAAEXZ 10008d64 f i pddpcie950:pddpcie950.obj
 0001:00007d84       ?Write_FCH@CMemRegpcie950@@UAAXE@Z 10008d84 f i pddpcie950:pddpcie950.obj
 0001:00007da8       ?Read_FCH@CMemRegpcie950@@UAAEXZ 10008da8 f i pddpcie950:pddpcie950.obj
 0001:00007dc8       ?Write_NMR@CMemRegpcie950@@UAAXE@Z 10008dc8 f i pddpcie950:pddpcie950.obj
 0001:00007dec       ?Read_NMR@CMemRegpcie950@@UAAEXZ 10008dec f i pddpcie950:pddpcie950.obj
 0001:00007e0c       ?Write_MDM@CMemRegpcie950@@UAAXE@Z 10008e0c f i pddpcie950:pddpcie950.obj
 0001:00007e30       ?Read_MDM@CMemRegpcie950@@UAAEXZ 10008e30 f i pddpcie950:pddpcie950.obj
 0001:00007e50       ?Write_485CR@CMemRegpcie950@@UAAXE@Z 10008e50 f i pddpcie950:pddpcie950.obj
 0001:00007e74       ?Read_485CR@CMemRegpcie950@@UAAEXZ 10008e74 f i pddpcie950:pddpcie950.obj
 0001:00007e94       ?Write_485DR@CMemRegpcie950@@UAAXE@Z 10008e94 f i pddpcie950:pddpcie950.obj
 0001:00007eb8       ?Read_485DR@CMemRegpcie950@@UAAEXZ 10008eb8 f i pddpcie950:pddpcie950.obj
 0001:00007ed8       ?Read_ID1@CMemRegpcie950@@UAAEXZ 10008ed8 f i pddpcie950:pddpcie950.obj
 0001:00007ef8       ?Read_ID2@CMemRegpcie950@@UAAEXZ 10008ef8 f i pddpcie950:pddpcie950.obj
 0001:00007f18       ?Read_ID3@CMemRegpcie950@@UAAEXZ 10008f18 f i pddpcie950:pddpcie950.obj
 0001:00007f38       ?WRITE_550_REGISTER@CMemRegpcie950@@UAAXPAEE@Z 10008f38 f i pddpcie950:pddpcie950.obj
 0001:00007f80       ?READ_550_REGISTER@CMemRegpcie950@@UAAEPAE@Z 10008f80 f i pddpcie950:pddpcie950.obj
 0001:00007fc8       ?WRITE_650_REGISTER@CMemRegpcie950@@UAAXPAEE@Z 10008fc8 f i pddpcie950:pddpcie950.obj
 0001:00007fe0       ?READ_650_REGISTER@CMemRegpcie950@@UAAEPAE@Z 10008fe0 f i pddpcie950:pddpcie950.obj
 0001:00007ff4       ?WRITE_950_REGISTER@CMemRegpcie950@@UAAXPAEE@Z 10008ff4 f i pddpcie950:pddpcie950.obj
 0001:0000800c       ?READ_950_REGISTER@CMemRegpcie950@@UAAEPAE@Z 1000900c f i pddpcie950:pddpcie950.obj
 0001:00008020       ?WRITE_ICR_REGISTER@CMemRegpcie950@@UAAXPAEE@Z 10009020 f i pddpcie950:pddpcie950.obj
 0001:00008038       ?READ_ICR_REGISTER@CMemRegpcie950@@UAAEPAE@Z 10009038 f i pddpcie950:pddpcie950.obj
 0001:0000804c       ??_ECMemRegpcie950@@UAAPAXI@Z 1000904c f i pddpcie950:pddpcie950.obj
 0001:0000804c       ??_GCMemRegpcie950@@UAAPAXI@Z 1000904c f i pddpcie950:pddpcie950.obj
 0001:00008080       ??0CPddpcie950@@QAA@PAGPAXPAU__HWOBJ@@@Z 10009080 f   pddpcie950:pddpcie950.obj
 0001:0000811c       ?SerialRegisterBackup@CPddpcie950@@UAAXXZ 1000911c f i pddpcie950:pddpcie950.obj
 0001:0000813c       ?SerialRegisterRestore@CPddpcie950@@UAAXXZ 1000913c f i pddpcie950:pddpcie950.obj
 0001:0000815c       ?ModemInterruptHandler@CPddpcie950@@UAAXXZ 1000915c f i pddpcie950:pddpcie950.obj
 0001:00008178       ?GetRxBufferSize@CPddpcie950@@UAAKXZ 10009178 f i pddpcie950:pddpcie950.obj
 0001:00008180       ?LineInterruptHandler@CPddpcie950@@UAAXXZ 10009180 f i pddpcie950:pddpcie950.obj
 0001:00008190       ??1CPddpcie950@@UAA@XZ     10009190 f   pddpcie950:pddpcie950.obj
 0001:000082b4       ?CreateHardwareAccess@CPddpcie950@@UAAHXZ 100092b4 f   pddpcie950:pddpcie950.obj
 0001:000083a4       ?XmitInterruptHandler@CPddpcie950@@UAAXPAEPAK@Z 100093a4 f   pddpcie950:pddpcie950.obj
 0001:000084ac       ??_GCPddpcie950@@UAAPAXI@Z 100094ac f i pddpcie950:pddpcie950.obj
 0001:000084ac       ??_ECPddpcie950@@UAAPAXI@Z 100094ac f i pddpcie950:pddpcie950.obj
 0001:000084d4       ??0CPddpcie950Isr@@QAA@PAGPAXPAU__HWOBJ@@@Z 100094d4 f   pddpcie950:pddisrpcie950.obj
 0001:0000851c       ??1CPddpcie950Isr@@UAA@XZ  1000951c f   pddpcie950:pddisrpcie950.obj
 0001:0000859c       ?Init@CPddpcie950Isr@@UAAHXZ 1000959c f   pddpcie950:pddisrpcie950.obj
 0001:000089e0       ?PeekEventData@CPddpcie950Isr@@IAAHPAE0@Z 100099e0 f i pddpcie950:pddisrpcie950.obj
 0001:00008a68       ?ReadEventData@CPddpcie950Isr@@IAAHPAE0@Z 10009a68 f i pddpcie950:pddisrpcie950.obj
 0001:00008ac4       ?EmptyEventData@CPddpcie950Isr@@UAAXXZ 10009ac4 f   pddpcie950:pddisrpcie950.obj
 0001:00008af8       ?WriteXmitData@CPddpcie950Isr@@IAAHE@Z 10009af8 f i pddpcie950:pddisrpcie950.obj
 0001:00008b68       ?ThreadRun@CPddpcie950Isr@@EAAKXZ 10009b68 f   pddpcie950:pddisrpcie950.obj
 0001:00008cd8       ?ReceiveInterruptHandler@CPddpcie950Isr@@UAAKPAEPAK@Z 10009cd8 f   pddpcie950:pddisrpcie950.obj
 0001:00008e84       ?CancelReceive@CPddpcie950Isr@@UAAKXZ 10009e84 f   pddpcie950:pddisrpcie950.obj
 0001:00008ed8       ?XmitInterruptHandler@CPddpcie950Isr@@UAAXPAEPAK@Z 10009ed8 f   pddpcie950:pddisrpcie950.obj
 0001:00009194       ?XmitComChar@CPddpcie950Isr@@UAAXE@Z 1000a194 f   pddpcie950:pddisrpcie950.obj
 0001:000092e8       ?CancelXmit@CPddpcie950Isr@@UAAHXZ 1000a2e8 f   pddpcie950:pddisrpcie950.obj
 0001:00009348       ?LineInterruptHandler@CPddpcie950Isr@@UAAXXZ 1000a348 f   pddpcie950:pddisrpcie950.obj
 0001:000093d8       ?ModemInterruptHandler@CPddpcie950Isr@@UAAXXZ 1000a3d8 f   pddpcie950:pddisrpcie950.obj
 0001:00009460       ?GetRxBufferSize@CPddpcie950Isr@@UAAKXZ 1000a460 f   pddpcie950:pddisrpcie950.obj
 0001:0000946c       ??_GCPddpcie950Isr@@UAAPAXI@Z 1000a46c f i pddpcie950:pddisrpcie950.obj
 0001:0000946c       ??_ECPddpcie950Isr@@UAAPAXI@Z 1000a46c f i pddpcie950:pddisrpcie950.obj
 0001:00009494       CreateBusAccessHandle      1000a494 f   ceddk:CEDDK.dll
 0001:000094a4       DDKPwr_RequestLevel        1000a4a4 f   ceddk:CEDDK.dll
 0001:000094b4       DDKPwr_ReleaseLevel        1000a4b4 f   ceddk:CEDDK.dll
 0001:000094c4       DDKPwr_GetDeviceLevel      1000a4c4 f   ceddk:CEDDK.dll
 0001:000094d4       DDKPwr_SetDeviceLevel      1000a4d4 f   ceddk:CEDDK.dll
 0001:000094e4       SetDevicePowerState        1000a4e4 f   ceddk:CEDDK.dll
 0001:000094f4       DDKPwr_Initialize          1000a4f4 f   ceddk:CEDDK.dll
 0001:00009504       DDKPwr_Deinitialize        1000a504 f   ceddk:CEDDK.dll
 0001:00009514       CloseBusAccessHandle       1000a514 f   ceddk:CEDDK.dll
 0001:00009524       WRITE_PORT_UCHAR           1000a524 f   ceddk:CEDDK.dll
 0001:00009534       READ_PORT_UCHAR            1000a534 f   ceddk:CEDDK.dll
 0001:00009544       MmMapIoSpace               1000a544 f   ceddk:CEDDK.dll
 0001:00009554       TranslateBusAddr           1000a554 f   ceddk:CEDDK.dll
 0001:00009564       WRITE_REGISTER_UCHAR       1000a564 f   ceddk:CEDDK.dll
 0001:00009574       READ_REGISTER_UCHAR        1000a574 f   ceddk:CEDDK.dll
 0001:00009584       MmUnmapIoSpace             1000a584 f   ceddk:CEDDK.dll
 0001:00009594       HalFreeCommonBuffer        1000a594 f   ceddk:CEDDK.dll
 0001:000095a4       BusTransBusAddrToStatic    1000a5a4 f   ceddk:CEDDK.dll
 0001:000095b4       HalAllocateCommonBuffer    1000a5b4 f   ceddk:CEDDK.dll
 0001:000095c4       ??2@YAPAXI@Z               1000a5c4 f   coredll:COREDLL.dll
 0001:000095d4       EventModify                1000a5d4 f   coredll:COREDLL.dll
 0001:000095e4       DisableThreadLibraryCalls  1000a5e4 f   coredll:COREDLL.dll
 0001:000095f4       LeaveCriticalSection       1000a5f4 f   coredll:COREDLL.dll
 0001:00009604       SetProcPermissions         1000a604 f   coredll:COREDLL.dll
 0001:00009614       EnterCriticalSection       1000a614 f   coredll:COREDLL.dll
 0001:00009624       InterruptDisable           1000a624 f   coredll:COREDLL.dll
 0001:00009634       InterruptDone              1000a634 f   coredll:COREDLL.dll
 0001:00009644       CloseHandle                1000a644 f   coredll:COREDLL.dll
 0001:00009654       Sleep                      1000a654 f   coredll:COREDLL.dll
 0001:00009664       WaitForSingleObject        1000a664 f   coredll:COREDLL.dll
 0001:00009674       CeSetThreadPriority        1000a674 f   coredll:COREDLL.dll
 0001:00009684       CeGetThreadPriority        1000a684 f   coredll:COREDLL.dll
 0001:00009694       memcpy                     1000a694 f   coredll:COREDLL.dll
 0001:000096a4       SetLastError               1000a6a4 f   coredll:COREDLL.dll
 0001:000096b4       SetThreadPriority          1000a6b4 f   coredll:COREDLL.dll
 0001:000096c4       LocalFree                  1000a6c4 f   coredll:COREDLL.dll
 0001:000096d4       DeleteCriticalSection      1000a6d4 f   coredll:COREDLL.dll
 0001:000096e4       InterlockedDecrement       1000a6e4 f   coredll:COREDLL.dll
 0001:000096f4       GetTickCount               1000a6f4 f   coredll:COREDLL.dll
 0001:00009704       InterlockedIncrement       1000a704 f   coredll:COREDLL.dll
 0001:00009714       InterlockedExchange        1000a714 f   coredll:COREDLL.dll
 0001:00009724       memset                     1000a724 f   coredll:COREDLL.dll
 0001:00009734       ExitThread                 1000a734 f   coredll:COREDLL.dll
 0001:00009744       CreateThread               1000a744 f   coredll:COREDLL.dll
 0001:00009754       InterruptInitialize        1000a754 f   coredll:COREDLL.dll
 0001:00009764       RegCloseKey                1000a764 f   coredll:COREDLL.dll
 0001:00009774       RegQueryValueExW           1000a774 f   coredll:COREDLL.dll
 0001:00009784       OpenDeviceKey              1000a784 f   coredll:COREDLL.dll
 0001:00009794       CreateEventW               1000a794 f   coredll:COREDLL.dll
 0001:000097a4       InitializeCriticalSection  1000a7a4 f   coredll:COREDLL.dll
 0001:000097b4       LocalAlloc                 1000a7b4 f   coredll:COREDLL.dll
 0001:000097c4       GetCurrentPermissions      1000a7c4 f   coredll:COREDLL.dll
 0001:000097d4       ResumeThread               1000a7d4 f   coredll:COREDLL.dll
 0001:000097e4       TerminateThread            1000a7e4 f   coredll:COREDLL.dll
 0001:000097f4       _purecall                  1000a7f4 f   coredll:COREDLL.dll
 0001:00009804       RegOpenKeyExW              1000a804 f   coredll:COREDLL.dll
 0001:00009814       CeEventHasOccurred         1000a814 f   coredll:COREDLL.dll
 0001:00009824       ??3@YAXPAX@Z               1000a824 f   coredll:COREDLL.dll
 0001:00009834       DDKReg_GetWindowInfo       1000a834 f   coredll:COREDLL.dll
 0001:00009844       wcstoul                    1000a844 f   coredll:COREDLL.dll
 0001:00009854       InterruptMask              1000a854 f   coredll:COREDLL.dll
 0001:00009864       _ultow                     1000a864 f   coredll:COREDLL.dll
 0001:00009874       wcslen                     1000a874 f   coredll:COREDLL.dll
 0001:00009884       RegSetValueExW             1000a884 f   coredll:COREDLL.dll
 0001:00009894       wcsrchr                    1000a894 f   coredll:COREDLL.dll
 0001:000098a4       wcsstr                     1000a8a4 f   coredll:COREDLL.dll
 0001:000098b4       CharUpperW                 1000a8b4 f   coredll:COREDLL.dll
 0001:000098c4       wcscpy                     1000a8c4 f   coredll:COREDLL.dll
 0001:000098d4       wcscat                     1000a8d4 f   coredll:COREDLL.dll
 0001:000098e4       wcsncpy                    1000a8e4 f   coredll:COREDLL.dll
 0001:000098f4       DDKReg_GetIsrInfo          1000a8f4 f   coredll:COREDLL.dll
 0001:00009904       KernelLibIoControl         1000a904 f   coredll:COREDLL.dll
 0001:00009914       FreePhysMem                1000a914 f   coredll:COREDLL.dll
 0001:00009924       NKDbgPrintfW               1000a924 f   coredll:COREDLL.dll
 0001:00009934       GetLastError               1000a934 f   coredll:COREDLL.dll
 0001:00009944       memchr                     1000a944 f   coredll:COREDLL.dll
 0001:00009954       __IMPORT_DESCRIPTOR_CEDDK  1000a954     ceddk:CEDDK.dll
 0001:00009968       __IMPORT_DESCRIPTOR_COREDLL 1000a968     coredll:COREDLL.dll
 0001:0000997c       __NULL_IMPORT_DESCRIPTOR   1000a97c     ceddk:CEDDK.dll
 0002:00000000       __imp_CreateBusAccessHandle 1000b000     ceddk:CEDDK.dll
 0002:00000004       __imp_DDKPwr_RequestLevel  1000b004     ceddk:CEDDK.dll
 0002:00000008       __imp_DDKPwr_ReleaseLevel  1000b008     ceddk:CEDDK.dll
 0002:0000000c       __imp_DDKPwr_GetDeviceLevel 1000b00c     ceddk:CEDDK.dll
 0002:00000010       __imp_DDKPwr_SetDeviceLevel 1000b010     ceddk:CEDDK.dll
 0002:00000014       __imp_SetDevicePowerState  1000b014     ceddk:CEDDK.dll
 0002:00000018       __imp_DDKPwr_Initialize    1000b018     ceddk:CEDDK.dll
 0002:0000001c       __imp_DDKPwr_Deinitialize  1000b01c     ceddk:CEDDK.dll
 0002:00000020       __imp_CloseBusAccessHandle 1000b020     ceddk:CEDDK.dll
 0002:00000024       __imp_WRITE_PORT_UCHAR     1000b024     ceddk:CEDDK.dll
 0002:00000028       __imp_READ_PORT_UCHAR      1000b028     ceddk:CEDDK.dll
 0002:0000002c       __imp_MmMapIoSpace         1000b02c     ceddk:CEDDK.dll
 0002:00000030       __imp_TranslateBusAddr     1000b030     ceddk:CEDDK.dll
 0002:00000034       __imp_WRITE_REGISTER_UCHAR 1000b034     ceddk:CEDDK.dll
 0002:00000038       __imp_READ_REGISTER_UCHAR  1000b038     ceddk:CEDDK.dll
 0002:0000003c       __imp_MmUnmapIoSpace       1000b03c     ceddk:CEDDK.dll
 0002:00000040       __imp_HalFreeCommonBuffer  1000b040     ceddk:CEDDK.dll
 0002:00000044       __imp_BusTransBusAddrToStatic 1000b044     ceddk:CEDDK.dll
 0002:00000048       __imp_HalAllocateCommonBuffer 1000b048     ceddk:CEDDK.dll
 0002:0000004c       \177CEDDK_NULL_THUNK_DATA  1000b04c     ceddk:CEDDK.dll
 0002:00000050       __imp_??2@YAPAXI@Z         1000b050     coredll:COREDLL.dll
 0002:00000054       __imp_EventModify          1000b054     coredll:COREDLL.dll
 0002:00000058       __imp_DisableThreadLibraryCalls 1000b058     coredll:COREDLL.dll
 0002:0000005c       __imp_LeaveCriticalSection 1000b05c     coredll:COREDLL.dll
 0002:00000060       __imp_SetProcPermissions   1000b060     coredll:COREDLL.dll
 0002:00000064       __imp_EnterCriticalSection 1000b064     coredll:COREDLL.dll
 0002:00000068       __imp_InterruptDisable     1000b068     coredll:COREDLL.dll
 0002:0000006c       __imp_InterruptDone        1000b06c     coredll:COREDLL.dll
 0002:00000070       __imp_CloseHandle          1000b070     coredll:COREDLL.dll
 0002:00000074       __imp_Sleep                1000b074     coredll:COREDLL.dll
 0002:00000078       __imp_WaitForSingleObject  1000b078     coredll:COREDLL.dll
 0002:0000007c       __imp_CeSetThreadPriority  1000b07c     coredll:COREDLL.dll
 0002:00000080       __imp_CeGetThreadPriority  1000b080     coredll:COREDLL.dll
 0002:00000084       __imp_memcpy               1000b084     coredll:COREDLL.dll
 0002:00000088       __imp_SetLastError         1000b088     coredll:COREDLL.dll
 0002:0000008c       __imp_SetThreadPriority    1000b08c     coredll:COREDLL.dll
 0002:00000090       __imp_LocalFree            1000b090     coredll:COREDLL.dll
 0002:00000094       __imp_DeleteCriticalSection 1000b094     coredll:COREDLL.dll
 0002:00000098       __imp_InterlockedDecrement 1000b098     coredll:COREDLL.dll
 0002:0000009c       __imp_GetTickCount         1000b09c     coredll:COREDLL.dll
 0002:000000a0       __imp_InterlockedIncrement 1000b0a0     coredll:COREDLL.dll
 0002:000000a4       __imp_InterlockedExchange  1000b0a4     coredll:COREDLL.dll
 0002:000000a8       __imp_memset               1000b0a8     coredll:COREDLL.dll
 0002:000000ac       __imp_ExitThread           1000b0ac     coredll:COREDLL.dll
 0002:000000b0       __imp_CreateThread         1000b0b0     coredll:COREDLL.dll
 0002:000000b4       __imp_InterruptInitialize  1000b0b4     coredll:COREDLL.dll
 0002:000000b8       __imp_RegCloseKey          1000b0b8     coredll:COREDLL.dll
 0002:000000bc       __imp_RegQueryValueExW     1000b0bc     coredll:COREDLL.dll
 0002:000000c0       __imp_OpenDeviceKey        1000b0c0     coredll:COREDLL.dll
 0002:000000c4       __imp_CreateEventW         1000b0c4     coredll:COREDLL.dll
 0002:000000c8       __imp_InitializeCriticalSection 1000b0c8     coredll:COREDLL.dll
 0002:000000cc       __imp_LocalAlloc           1000b0cc     coredll:COREDLL.dll
 0002:000000d0       __imp_GetCurrentPermissions 1000b0d0     coredll:COREDLL.dll
 0002:000000d4       __imp_ResumeThread         1000b0d4     coredll:COREDLL.dll
 0002:000000d8       __imp_TerminateThread      1000b0d8     coredll:COREDLL.dll
 0002:000000dc       __imp__purecall            1000b0dc     coredll:COREDLL.dll
 0002:000000e0       __imp_RegOpenKeyExW        1000b0e0     coredll:COREDLL.dll
 0002:000000e4       __imp_CeEventHasOccurred   1000b0e4     coredll:COREDLL.dll
 0002:000000e8       __imp_??3@YAXPAX@Z         1000b0e8     coredll:COREDLL.dll
 0002:000000ec       __imp_DDKReg_GetWindowInfo 1000b0ec     coredll:COREDLL.dll
 0002:000000f0       __imp_wcstoul              1000b0f0     coredll:COREDLL.dll
 0002:000000f4       __imp_InterruptMask        1000b0f4     coredll:COREDLL.dll
 0002:000000f8       __imp___rt_sdiv            1000b0f8     coredll:COREDLL.dll
 0002:000000fc       __imp___rt_udiv            1000b0fc     coredll:COREDLL.dll
 0002:00000100       __imp__ultow               1000b100     coredll:COREDLL.dll
 0002:00000104       __imp_wcslen               1000b104     coredll:COREDLL.dll
 0002:00000108       __imp_RegSetValueExW       1000b108     coredll:COREDLL.dll
 0002:0000010c       __imp_wcsrchr              1000b10c     coredll:COREDLL.dll
 0002:00000110       __imp_wcsstr               1000b110     coredll:COREDLL.dll
 0002:00000114       __imp_CharUpperW           1000b114     coredll:COREDLL.dll
 0002:00000118       __imp_wcscpy               1000b118     coredll:COREDLL.dll
 0002:0000011c       __imp_wcscat               1000b11c     coredll:COREDLL.dll
 0002:00000120       __imp_wcsncpy              1000b120     coredll:COREDLL.dll
 0002:00000124       __imp_DDKReg_GetIsrInfo    1000b124     coredll:COREDLL.dll
 0002:00000128       __imp_KernelLibIoControl   1000b128     coredll:COREDLL.dll
 0002:0000012c       __imp_FreePhysMem          1000b12c     coredll:COREDLL.dll
 0002:00000130       __imp_NKDbgPrintfW         1000b130     coredll:COREDLL.dll
 0002:00000134       __imp_GetLastError         1000b134     coredll:COREDLL.dll
 0002:00000138       __imp_memchr               1000b138     coredll:COREDLL.dll
 0002:0000013c       \177COREDLL_NULL_THUNK_DATA 1000b13c     coredll:COREDLL.dll

 entry point at        0001:00000ac0

 Static symbols

 0001:00002288       SerialDispatchThread       10003288 f   mddpcie950:mddpcie950.obj
